:020000040000FA
:0200000077285F
:08000800FE00030E8301C60097
:100010000A08C7008A016E288207083402340834AF
:10002000503400340F340834023420345034003457
:100030000434083402342034503400340434053499
:10004000053420345034003404340534053420346D
:1000500008340234203402340834203408340234A2
:10006000203402340834203450340034043405344D
:10007000053420345034003404340534053420343D
:100080000834023420340234083420340834023472
:10009000203402340834203450340034043408341A
:1000A00002340834503400340F340834023420341D
:1000B00050340034043408340234203450340034D2
:1000C00004340830C8000310C20D0310C00D031C17
:1000D0006B284108C207C80B632808004808C900FC
:1000E0004008C3004108C4004208C5009229831695
:1000F00085120512851005107D107D08831285007C
:10010000CF298312121187309205FC301205023874
:1001100092005D30831692008312D901D501083018
:10012000D7000230D6000830D8005A14FD167D08DA
:1001300085007D167D0885008C1083168C140800C0
:100140007D127D088500121508001211FD167D082C
:1001500085007D167D08850008008C1C33298C10D5
:10016000FD147D0885005A1CEF2858080319F22851
:1001700057080319C028FD167D088500D703C72836
:1001800056080319C728FD127D088500D6035708B5
:10019000CC15031DCC1156084C16031D4C12CC1661
:1001A000CC194C1ECC12CC1EF228D8035508C00026
:1001B0000330C100612083124208CA0000308A0067
:1001C0004A080C208312D7004208CA004A0ACB0012
:1001D00000308A004B080C208312D600F228FD1252
:1001E0007D088500D90A50305902031D3029D901F4
:1001F0005A1CFC285A10FD285A145A1C3029580839
:10020000031D1829D50A1C3055020319D5015508BC
:10021000C0000330C100612083124208CA000230CE
:100220004A07CB0000308A004B080C208312D8000C
:100230005508C0000330C100612083124208CA0083
:1002400000308A004A080C208312D7004208CA00F6
:100250004A0ACB0000308A004B080C208312D600DB
:10026000FD107D0885004308C0004408C100450812
:10027000C2004908C80047088A00460E8300FE0EE7
:100280007E0E0900103083169F00953083129F0068
:100290005A11991319120C1383160C1708004E10DB
:1002A0000C1F572983160C1F572983124E148312D3
:1002B0004E1CAD285A1973291E08C000FF30C1001A
:1002C000612083124208CA00CB0183161E088312E4
:1002D000CC00CD014D084B07D0004C084A07CF0099
:1002E0000318D00A5A150C13AD2883125A1D7F2902
:1002F0004F08D1005008D2005A1140140800401095
:10030000080083129F14080083125A1195309F0031
:100310000800803083129F0008008B100B16831298
:10032000DA1008008B1C4F298B10DA144F29A020FB
:10033000842183120313AD30C000E630C1000A12DD
:100340008A11C10B9F290A128A11C00B9D29000036
:10035000000000000000000000000000000000009D
:10036000D301D401DA100800A520892183120313D8
:10037000AD30C000E630C1000A128A11C10BBC29A1
:100380000A128A11C00BBA29000000000000000008
:1003900000000000000000000000630097298312A5
:1003A0000313AD30C000E630C1000A128A11C10B40
:1003B000D5290A128A11C00BD329000000000000C1
:1003C00000000000000000000000000083169F01F4
:1003D00083129F019A019C01422181208D21831269
:1003E000D301D4010B178B17B42175218312DA11B5
:1003F0004018DA15DA1D102A01305202031D022AB4
:100400001830510203190F2A031C0F2A0A30530215
:10041000031D0D2AD301B421102AD30A102AD301B7
:100420008312DA1C1C2A05305402031D1A2AD40137
:10043000B4211D2AD40A1D2AD40181218312031359
:100440009330C0001A30C1000A128A11C10B242A4D
:100450000A128A11C00B222A0000000000000000CE
:040460000000F5297A
:02400E00443C30
:00000001FF
